:0200000097283F
:08000800E02A0D340A345034E3
:10001000433420344C34413420342D34203456348D
:10002000653472342E34203430342E34313431344B
:1000300000340D340A344E3475346D342034743445
:100040006F342034773472346934743465343A341C
:1000500000340D340A3464346F346E3465340D3436
:100060000A3400340D340A3445346E347434653443
:1000700072342034733469347A3465343A34003459
:100080000D340A34533469347A3465343D340034E1
:100090000D340A3445346E3474346534723420348B
:1000A00063346C346B343A3400340D340A344334E2
:1000B0006C346B343D3400340D340A3453347434AE
:1000C0006F34723469346E3467342E342E342E34E7
:1000D000203400340D340A3445346E3474346534BD
:1000E0007234203474347234693467343A340034EE
:1000F0000D340A345434723469346734203464342F
:1001000069347334613462346C346534643421345A
:1001100000340D340A34573461346934743469342A
:100120006E3467342E342E342E3420340034F401EF
:10013000B922EF220423871105300B230D3026232B
:100140000A3026233A302623741CA428741075081C
:10015000643C03195A2A7508773C0319202A75084C
:10016000733C0319BC297508633C0319772975088A
:10017000723C031990297508743C03192E297508DF
:100180006C3C0319C428A428831203136A300B2380
:10019000741CC828741075081B3C03199E28750828
:1001A000303C03192A29FA01FB01FC0120302623E7
:1001B0000830F600741CDA28741075081B3C03190B
:1001C0002A297508303C0319F2287508313C0319B7
:1001D000EE287508783C0319F028DA287A14F228FA
:1001E0007C14F228F60BF528FA280310FA0D0310F8
:1001F000FC0DDA28FC09203026230830F600741C98
:10020000FF28741075081B3C03192A297508303C17
:10021000031912297508313C031910297508FF28A4
:100220007B141229F60B152918290310FB0DFF2842
:1002300079143A302623203026237A089A22203057
:1002400026237B089A22203026237C089A222930F4
:100250000B239E28791078300B239E2883160313D6
:10026000FF308600831203138714071107128711CA
:10027000791C642989300B23203026233130262332
:1002800074184A2906087C057A060319502987152F
:1002900087114029750874101B3C031D40296A29E9
:1002A000203026233230262374185E2906087C0568
:1002B0007B06031964298715871154297508741062
:1002C0001B3C031D3A296A295C300B2374187129E1
:1002D000871E6629871507160715871029300B23F7
:1002E0009E28750874101B3C031D66296A29831219
:1002F000031348300B23741C7B29741075081B3CB6
:1003000003199E2830307502F600073C031C9E2816
:1003100076080739890055300B23750826239E2857
:10032000071587150714071007140710071407107F
:100330000714071007140710871107140710060881
:100340002623071407107418B629871E9D298715C0
:1003500007140710071407100714071007140710D5
:1003600007140710871129300B239E287410750875
:100370001B3C031DA529A7298312031332300B232D
:10038000741CC029741075081B3C03199E2875083D
:10039000303C0319E8297508313C0319EF29750829
:1003A000323C0319F6297508333C0319FD297508F9
:1003B000343C0319042A7508353C03190B2A7508C7
:1003C000363C0319122A7508373C0319192A9E284E
:1003D00040300B2330302623003085009E284030EB
:1003E0000B2331302623043085009E2840300B2318
:1003F00032302623103085009E2840300B233330C6
:100400002623143085009E2840300B2334302623C9
:10041000203085009E2840300B23353026232430A1
:1004200085009E2840300B2336302623303085004F
:100430009E2840300B2337302623343085009E28F9
:10044000831203135730A20719300B2383120313AF
:1004500022089A220D3026230A302623071107147A
:100460000710871507140710071407100714071043
:100470008711831603138601831203132208860053
:1004800007140710871E402A83160313FF308600C7
:100490008312031307158715071407100714071095
:1004A00007140710071407100714071087112930C5
:1004B0000B239E28831203131A30A0001630A100CC
:1004C0000D3026230A30262387150714071007143A
:1004D00007100714071007140710071407108711D7
:1004E0000714071006089A2220302623A00B932A0F
:1004F0000D3026230A302623831203131A30A0005E
:10050000A10B932A741C822A741075081B3C0319D2
:100510009E287508203C031D822A1630A1000D304C
:1005200026230A30262307140710871E702A293035
:100530000B239E2883120313F700F039F8000310F1
:10054000F80C0310F80C0310F80C0310F80C0A3028
:100550007802303003183730780726230F307705BC
:10056000F8000A3078023030031837307807262335
:100570000800831603130B308500FF308600E0303F
:100580008700FF3088000030890004309F0083120C
:100590000313F90100308900003085000716871029
:1005A00007158715071007140710071407100714FD
:1005B0000710071407100714071007140710080086
:1005C000F200030E8301F300FF22F5008C12741475
:1005D0002623EF22730E8300F20E720E090083169B
:1005E00003130C309900181518128312031398176F
:1005F0001816831603138C168312031308008C1E1F
:10060000FF2A1A0818120800831603130B178B17FA
:10061000831203130800F1001523F0007008031D76
:10062000122B08002623F10A0C2B71088200831676
:1006300003130C309900181518128312031398171E
:1006400018168C1E212B1A08181208008316031383
:10065000981C282BF0000C309900181518128312E2
:100660000313981783160313981670088312031345
:0406700099000800E5
:02400E00313D42
:00000001FF
